:020000020000FC
:100000005CCDA4C1000000001FC000008DC0000036
:10001000000097C00000000000000000020304067A
:10002000080C10182030406080000406080C1018DE
:100030002030406080A0C0000003070F1F000505AE
:100040000D050305030302004FB662FD0CC05520E9
:1000500041F00994C52DC095089483FDC795C4BD92
:1000600064604FBE1895C0916400089483FDC795E5
:10007000C4BD6B7FC0916400CF3F09F41EC070FF08
:100080001AC082FD05C04FBE9598AC98C0981895CF
:1000900076FD0EC064FD0CC0C091B100C0FD949807
:1000A000C1FDAD98C2FDAB98CAEFC095CA95F1F7F6
:1000B0009598AC98C0984FBE189524BCCC27C064C6
:1000C000C8BF6460F8CFC6CF70FFC4CF64FDC2CF95
:1000D000959AC0CF70FFBECF64FDBCCFAC9ABACFAB
:1000E00070FFB8CF64FDB6CFC09AB4CF949A70FFBA
:1000F000B1CF64FDAFCFC7E0CA95F1F7959AAACF0B
:10010000AD9A70FFA7CF64FDA5CFC7E0CA95F1F700
:10011000AC9AA0CFAB9A70FF9DCF64FD9BCFC7E098
:10012000CA95F1F7C09A96CF4FB6C9B7CF7EC9BF6F
:100130006E7FCCB5CE0DDDB5DF1DDBBDCABD4FBEBC
:1001400018953FB68F7EABB7A074A2118061A0E076
:10015000ABBFA9B7AE7FA9BF7894A0916800AA23CE
:1001600041F085FD2EC0A0916800AA95A09368007B
:1001700028C040E050E085FD14C0A0B396FDA095D6
:10018000A2FD4FEFA3E096FDA2E0A5BFAA27A064C1
:10019000AABF8D7FA0B396FDA095A2FD5FEF451786
:1001A00041F7A8E161FDA093680085FD03C0A8E1C7
:1001B000A0936800409396008160442311F0209240
:1001C000990085FD0EC0A0916900AA2331F0A0918D
:1001D0006900AA95A093690004C08061AA27A06461
:1001E000AABF80FF3DC0A09196004A2F61FF8E7F7D
:1001F00085FD18C0403F08F040EFA42FA295AF70D6
:100200004A0F5091B600533069F0A695A69550FD5F
:1002100001C0A69552FD03C0A41B4A2F03C04A0F7C
:1002200008F44FEFA0919F004A1708F44A2F40931B
:100230006100A72FA670A1F073FD12C0A0917000FD
:10024000AA0FAA0F50919E0056955695541708F084
:10025000452F4A0F4093610018F4AFEFA09361005F
:10026000A0916100A093630040916300A0919B0066
:100270004A1708F04A2F542EA091A000AA2309F48F
:1002800022C0542F5A1B10F4A42F50E0BA2E889489
:10029000AA1FAA2EA091A200A095AA22A50E58F0EE
:1002A000A091A100A21509F0AA95AA0EA093A10001
:1002B00048F04A2D08C0A091A100BA1608F0A395F5
:1002C000A093A1004FEF409364007F7B485F08F04C
:1002D0007064A0916000A395A093600051F0F89421
:1002E000A9B7A160A9BF84FF02C0A0E4ABBF3FBE15
:1002F0001895A0917400A395A093740041E05091CB
:100300006800552329F085FF03C05A955093680073
:10031000A0919600A13018F0209299000DC0209273
:100320009A002092A300A0919900AF5FA09399003A
:1003300018F0AFEFA0939900F894A9B7A160A9BFF6
:1003400084FF02C0A0E4ABBF3FBE18953FB64CB5DA
:100350005DB58F7EABB7A074A2118061A0E0ABBF8A
:10036000A9B7AE7FA9BF789481FD23C0A2E096FD16
:10037000A3E0A5BF8260A0B396FDA095A2FF05C033
:1003800040936500509366003EC1A3E096FDA2E055
:10039000A5BFAA27A064AABF8D7F85FF01C026C183
:1003A00040E0A0B396FDA095A2FD20C14093960029
:1003B0000FC1A3E096FDA2E0A5BF8D7F61FF71C0D4
:1003C000A2E096FDA3E0A5BFAA27A064AABF826011
:1003D0004093910050939200A0908F004A19B090E2
:1003E00090005B09BB24A22C4C38520518F42092D3
:1003F000950049C0A091D400AA2359F1483C520568
:1004000028F4A0E1BA2EAAE0AA2E23C04836A1E023
:100410005A0728F4A8E0BA2EAFE0AA2E1AC0403D31
:10042000A2E05A0728F4A4E0BA2EAEE1AA2E11C029
:10043000403AA5E05A0728F4A2E0BA2EACE3AA2E6F
:1004400008C04839A8E05A0720F4A1E0BA2EA8E76E
:10045000AA2EC42EA0919300CA1AD52EA091940062
:10046000DA0ADD202AF4AFEFC094D094CA1ADA0A6F
:1004700020929500A8E0A210A0E0CA14DA0618F4B1
:10048000A1E0A09395004093930050939400409175
:1004900091005091920040938F005093900042E061
:1004A00097C0A09165004A1BA09166005A0B94FD6D
:1004B00082C093FD80C092FD7CC086FF03C0D52E14
:1004C000C42E0CC05695479591FD73C0569547951F
:1004D00090FD6FC0D52EC42ED694C79461FD19C06F
:1004E000AC2DAC51AD2DA24008F005C0DD2089F443
:1004F000AC2DA85C70F4A0916700A395AA2311F01D
:10050000A0936700AA3008F471C020929600816021
:100510006DC0A0916700AA2319F0AA95A093670067
:10052000A22C5091BA0097FD06C0A090C80053308D
:1005300011F4A090D000AAEFAA0EA22DA21DCA18F5
:10054000DA0A4FB74170533049F4442321F087FD54
:1005500005C0806803C087FF01C08F77442359F02E
:10056000533031F4AFEFC094D094CA1ADA0A03C002
:1005700040E050E020C0533049F4CC0CDD1CAAE030
:10058000CA1AD20818F4A0E0CA2ED22CAFEFCA16AD
:10059000D20418F04FEF50E00EC0A091AC00CA9EFC
:1005A000412D000C441F50E008F012C04FEF50E006
:1005B0000FC05695479594FF07C0552309F04FEF9C
:1005C000A42FA6954A0F521D4F3F520508F04FEF3A
:1005D00040939600816061FF09C0AFE1A095A92317
:1005E000AB299A2F8F7DBB2009F48062A8E1A093EC
:1005F000680085FF03C0AAE0A093680061FD03C006
:1006000085FD01C08F7E85FD03C0A6E0A093690033
:10061000F894A9B7A160A9BF84FF02C0A0E4ABBF52
:100620003FBE189511E00AC013E008C01AE006C0EA
:100630001EE104C014E602C018EC00C005E1BB27AF
:10064000BA95F1F70A95D9F71A95C1F708952AE3F3
:1006500038E709C020E33CE806C02AE234EB03C0D7
:1006600025E238EC00C0B091AD00BA9509F40895C8
:1006700012E0BB27AD9ABA95F1F7AC9ABA95F1F7AB
:10068000AC98BA95F1F7AD98BA95F1F7123009F038
:10069000959A123009F4C09AB091AD00BA95F1F76D
:1006A000123009F09598123009F4C098B7E8BA955D
:1006B000F1F71A95F1F6022FB22FBA95F1F70A95D4
:1006C000D9F73A9581F6AD9A0895221B39E0001FBB
:1006D0003A9509F40895221F211B18F4210F8894DC
:1006E000F6CF0894F4CF622C722CB0E08894B395C6
:1006F000221F331FE0F7379527958894912E802E7F
:10070000020B130B10F4192D082D10F4889401C05E
:100710000894661C771CBA9571F7172D062D08955D
:10072000322D11232AF43A9500951095031B130BD3
:10073000F894029F712C002D129F912C802C78949C
:10074000780C172D921C292DB4E06B2E2695179549
:1007500007956A94D9F7332321F000951095031B70
:10076000130B0895089510917B00169500917A005F
:100770000795B0917E00B01B0B2FB0917F00B10B9D
:100780001B2F28F40038BFEF1B0740F009C00F37BC
:10079000120508F405C00FE710E002C000E81FEFE3
:1007A0000093830010938400089500918300B0911A
:1007B00080000B0F10918400B09181001B1F20E07E
:1007C0003091840033230AF42A95B09182002B1FC4
:1007D0001AF4203F40F00AC02F3008F407C00FEF92
:1007E0001FEF2FE003C000E010E020EF3091630026
:1007F000B0919B003B1718F4323030F009C0B09133
:100800008400BB235AF004C0B0918400BB2332F4AF
:10081000009380001093810020938200089520911E
:10082000D70000918300000F10918400111F78DF22
:1008300011232AF40038BFEF1B0740F009C00F371F
:10084000120508F405C00FE710E002C000E81FEF32
:10085000002352F0B0916200B01B0B2F18F0013052
:1008600008F00AC001E008C000950F5FB091620077
:100870000B0F08F001C00FEF009385000895209141
:10088000D80000918100109182004ADF11232AF4E0
:100890000130BFEF1B0740F009C00F3F120508F4FD
:1008A00005C00FEF10E002C001E01FEF112352F06E
:1008B000B0918500B01B0B2F18F0013008F00AC072
:1008C00001E008C000950F5FB09185000B0F08F0A4
:1008D00001C00FEF0093630008950FEF71FD1EC07C
:1008E000B091D300BB23D1F0B0917B00BB23B1F01A
:1008F0000FEF10917B00E9DEF894B091730072FD68
:10090000B5E00B9F112D002D7894112309F00FEF06
:10091000B0919E000B1710F400919E0000939D0073
:10092000089500917A0010917B0000541140B0911D
:100930009D0010F4BA9501C0B39511F0B0939D00DD
:10094000089500C008952091B500B6B1B6FDFBCF63
:1009500004B115B1B6B1BF77B6B9B091AA00B395DD
:10096000B093AA00B83060F12092AA00B091D200F2
:10097000BB2321F1112329F0B091AB00BF3F61F0FF
:1009800009C0B091AB000B1739F020F4BB2321F064
:10099000BA9502C0B395E1F300919B00B093AB0010
:1009A000B83850F400ECBD3738F400E8B23720F422
:1009B00000E4B73608F400E000939B007F7E0895C2
:1009C000B0919B00B39511F0B0939B00B091AA0039
:1009D000B73009F47061089502E3F894B091D9003A
:1009E0000B9F012D000C001F7894B0919B000B17FA
:1009F00010F000919B000093610000936300502E63
:100A00000093640000939E00089520927A00B0EF56
:100A1000B0937B000895F8940CB51DB52091740037
:100A20007894309175006090760000937500109373
:100A30007600031B160971FD03C077FD80C028C036
:100A400070907700209377002709222319F00FEF89
:100A50001FEF0EC08090780090907900309378005E
:100A600060927900009175001091760008191909BB
:100A700020917A0030917B0036952795020F131F45
:100A800010F40FEF1FEF00937A0010937B002BC040
:100A900020917A0030917B003901B4E08B2EB2E0D6
:100AA0009B2E343040F08A949A94383020F072FDB6
:100AB00002C08A949A94769467948A94E1F72619EE
:100AC0003709992021F0169507959A94E1F7200FA0
:100AD000311F20937A0030937B0028F43FEF30934E
:100AE0007A0030937B00323008F4706871FF02C0E6
:100AF000B3E00DC0B091C40000917100023838F02D
:100B0000B395003A08F0B395B63008F0B5E09B2EE7
:100B1000B4E08B2E10917B0000917A0024E01695B2
:100B200007952A95E1F70819120928F0B02FB2505D
:100B3000B12FB20910F402E010E0980126C0209114
:100B40007A0030917B0039017694679466946694BC
:100B500066942619320906950695200F321D2093BA
:100B60007A0030937B00323008F07F7704E03695CE
:100B700027953695279526952695201B10F022302F
:100B800008F422E089019090C40060FDFECFE0905F
:100B90008B00F0908C006160B9B7B061B9BF3801CB
:100BA00077FD41C07694679400938B0010938C007E
:100BB000B92DB330E1F0B0FD04C0060D171D93014F
:100BC00006C0000F111F0250120922E030E0B92DBB
:100BD000B33068F020938D0030938E00009387002F
:100BE000109388006092890070928A003AC0009346
:100BF0008D0010938E0020938700309388006092C0
:100C0000890070928A0071FF0DC0BFE0B0938D0023
:100C100020928E00B093890020928A00B0938B00BE
:100C200020928C001EC0669400938B00B92DB330C7
:100C300091F0B0FD03C0060D262D03C0000F025039
:100C400022E0B92DB33038F020938D000093870057
:100C50006092890006C000938D0020938700609207
:100C6000890000917C0002FD0350013029F495FDBC
:100C70000AC0B6E0B7B909C0023019F4B7E0B7B995
:100C800004C095FDF6CFB0E0B7B90091A200000F07
:100C900010F4BBE60B270093A20060FDFECFB2E08C
:100CA000B0936E006160B9B7B061B9BFB72FB670CD
:100CB000D1F020917A0030917B00369527953695BA
:100CC000279571FF02C0B0E43B0FF8940CB51DB539
:100CD000020F131F1BBD0ABD6160B0E1B8BFB9B7F9
:100CE000B061B9BF78940895686020927D0020E0DB
:100CF00066FD20E206C0686020927D0020E266FD6D
:100D000020E001E011E077FD11C0B72FB67009F0C7
:100D1000677F14E100917B00069509F403950F307D
:100D200008F00FE071FF02C004E114E160FD0FC0A4
:100D3000B0917D00BB2359F071FF06C0B0916E00E9
:100D4000BA95B0936E0011F470624FC0ABDFB0B7CC
:100D5000B77FB0BFB8B1B0B7B860B0BFB0917D00D9
:100D6000B395B0937D00B8B177FD06C0B1E071FDD9
:100D7000B3E0BA95F1F7B8B1B072B21709F02AC072
:100D800071FF05C00395011708F00A95CFCF63FDE9
:100D900005C00395011708F0B4CFC8CF677FF8945A
:100DA0003CB56DB470907A00B0917B00770CBB1F9E
:100DB00008F4BFEF770CBB1F08F4BFEF370D6B1EB5
:100DC0006BBC3ABD6160B0E1B8BFB9B7B061B9BF43
:100DD000789497CFB0916D00B13008F492CF63FD55
:100DE00090CF0A9509F0A2CF7F7D20918D003091A0
:100DF0008E00F894B0E1B8BF0CB51DB5020F131FFB
:100E00001BBD0ABDE0908700F09088006160B9B713
:100E1000B061B9BF7894B72FB67039F0B0916D005A
:100E200072FFB395B0936D0009C075FF07C066FDF2
:100E300005C063FD03C0BF91BF91F7C4089500E0F2
:100E400063FF01C001E0F89410917100B7E01B9FAF
:100E5000212D102D7894200F2695179526951795FE
:100E60002695179510937100183718F4B8E7B093CA
:100E7000710000917100B09172000B1720F0606159
:100E80009598AC98C09860FDFECFE0908900F090F6
:100E90008A006160B9B7B061B9BF0895B2E095FD4D
:100EA0000AC0F894B0937C00AD9A949862FF01C098
:100EB000C09A7894F4C0F894B0937C00AD9AAB9843
:100EC00062FF01C0959A7894EAC0B3E082FF24C023
:100ED00095FD11C002E0F894B0937C00E0E8F0E0EA
:100EE0000093B100C098AB9A62FF02C0AC9A01C0F7
:100EF000AD987894D4C002E0F894B0937C00E0E818
:100F0000F0E00093B1009598949A62FF02C0AC9A09
:100F100001C0AD987894C3C095FD0BC0F894B09310
:100F20007C00EAE6F0E0C09862FF01C0AC9A7894D9
:100F3000B6C0F894B0937C00EAE6F0E0959862FFC2
:100F400001C0AC9A7894ABC0B4E095FD0AC0F894A7
:100F5000B0937C00949AAB9862FF01C0AC9A7894ED
:100F60009EC0F894B0937C00AB9A949862FF01C045
:100F7000AC9A789494C0B5E082FF24C095FD11C06E
:100F800001E0F894B0937C00E6E7F0E00093B10054
:100F9000AC98AD9A62FF02C0959A01C0949878947B
:100FA0007EC004E0F894B0937C00EAE8F0E000939F
:100FB000B100AC98AD9A62FF02C0C09A01C0AB9874
:100FC00078946DC095FD0BC0F894B0937C00E4E676
:100FD000F0E0AC9862FF01C0959A789460C0F894F4
:100FE000B0937C00E0E7F0E0AC9862FF01C0C09AEB
:100FF000789455C0B6E095FD0AC0F894B0937C0093
:10100000AB9AAD9862FF01C0959A789448C0F89465
:10101000B0937C00949AAD9862FF01C0C09A789416
:101020003EC0B1E082FF24C095FD11C004E0F894F9
:10103000B0937C00EAE8F0E00093B1009598949AB0
:1010400062FF02C0C09A01C0AB98789428C001E04A
:10105000F894B0937C00E6E7F0E00093B100C0980C
:10106000AB9A62FF02C0959A01C09498789417C019
:1010700095FD0BC0F894B0937C00E0E7F0E0959804
:1010800062FF01C0C09A78940AC0F894B0937C00C3
:10109000E4E6F0E0C09862FF01C0959A78946F7E14
:1010A000089523E630E0F9012092B1009598AC98BC
:1010B000C098949AAD9AAB9A6B7F0895A2EBB0E07A
:1010C0000FEF0D930D930D930D9303E00D9304E03B
:1010D0000D930BE00D9303E00D9301E00D9301E000
:1010E0000D93AEEBB0E001E00D930FEF0D930D9378
:1010F0000D930D930D9303E00D930FEF0D930FEFF1
:101100000D930D9305E20D9300ED0D930AEF0D93F2
:101110000AEF0D9304E00D930FEF0D9301E00D9393
:1011200000E00D930AE70D930FEF0D9300E00D9390
:1011300001E00D9300E00D9303E00D9300E00D93AB
:1011400008952091B9008B7F233009F48460B09119
:10115000BA00B33019F09F7DB1FD90629F7BB091D2
:10116000BB00B1FD9064223011F0886001C0877F20
:1011700008950A95E00FF21DB4910895ECE1F0E0B6
:101180000091B200F6DFB093D700ECE1F0E00091FF
:10119000B300EFDFB093D800EAE2F0E00091B800CE
:1011A000E8DFB093D9000091B800023008F402E003
:1011B00000937300B091CE000FEFB23009F400EA53
:1011C000B33009F402E800937200E8E3F0E0009124
:1011D000D500CFDFB093A000089508952091C800F6
:1011E0003091C900B091BA00B33009F43E5097FF76
:1011F00002C020E03FEFB32FB21B6B2EB25810F4A9
:10120000B2E86B2E00E00395609EB12DBD57D8F378
:101210000093AC0008959068E1DF0ADA09DA20E073
:1012200030E0B0E16B2E00DAB09196002B0F321D4A
:101230006A94C9F7B4E036952795BA95E1F7822EFE
:101240009F77CCDF0895F894E3E0F0E0B9E0B7BF12
:10125000B491B078C1F3F894A895B1B5B861B1BDB7
:10126000B0E0B1BDB4E0BEBFBFE5BDBF1ADFB0E0C6
:10127000B8BBB1E1B7BBB8E2B5BBB8E3B4BBB0E152
:10128000B2BBB0E3B1BB2224A0E0B0E02D92AA3102
:10129000E9F7A0E6B0E00FEF2D920A95E9F7B1E08B
:1012A000B093A2000BDFF9D2B6B1B460B6B9009129
:1012B000CA000093AD00B1E0B0936A00F894BCD9C5
:1012C000C6D9B6D9C7D9B4D9C8D9B2D96DD3B4D9CA
:1012D000B3D9B0D9F8940AEF1AEFA0B396FDA09550
:1012E000A2FF1FC01A95C9F70A95B1F7E0E0FCE12B
:1012F000B591B43E39F4B591B03E21F4B591BF3FFC
:1013000009F40CC0E0E0F395F395B591B83F49F4CA
:10131000B591B43931F4B591BA3A19F4EE27F6958E
:1013200009940FDF2BDF59DF59DF0091CA000093CA
:10133000AD00B7DEB2E0B3BFB2E0BEBDB2E0B5BD56
:10134000B1E5B8BFB9BFB0B7B77FB0BFB8B1B0B73C
:10135000B860B0BF67D97894F4DA20927000B3E037
:1013600096FDB2E0B5BFB0E4BBBFBB27B064BABF67
:101370008D7F62D9626033E02CE0B0919500BB2391
:1013800021F42CE03A9509F4A5CF52D980FFA2CFE1
:101390008E7FB0919600B23078F3B92FBF71009173
:1013A000980000939700B0939800B01729F72A95FA
:1013B00021F76D7FB3E096FDB2E0B5BFBB27B06407
:1013C000BABF8D7FB091D400BB2321F48062B92FC6
:1013D000B0709B2F8F7B209267002CD985FF05C0B2
:1013E000B0916700BA3008F080641ED902E085FF32
:1013F00001C000E0B0919600B017B8F3F89427D977
:1014000026D925D9789418D920928600B091BA00AF
:10141000B33009F47EC008D9B091BE00B13008F4F1
:1014200078C0B0916A00B13008F473C085FD18C06F
:10143000B0919600BF3F08F46CC0F89411D978942D
:10144000F9D8B0919600B130C0F7F89400D9EED831
:10145000FED87894EFD8B0919600BF3FB0F3D6C2D3
:10146000B8E09B2E9068F894B9DE7894E3D8F894AD
:101470009F77B4DE80909600B0919600BF37789445
:1014800008F44FC0CFD8F894EBD878949A9451F7D9
:10149000C2DEB82DB550B093C900CED8F89489D229
:1014A0007894BAE09B2E9068F89498DE7894C2D82D
:1014B000F8949F7793DE80909600B0919600BF37A6
:1014C000789478F7AFD8F894C2D8B0D8C0D87894C8
:1014D0009A9449F7A0DEB82DBB5FB093C8000B2FDC
:1014E0001091C900125810F0100B20F4B2E80B0F45
:1014F0000093C900A1D8F894FDD16AD278949AD803
:10150000F8946CDE7894B0919600BF3F08F48ECFCB
:101510007DC200919600B09186000B1710F00093E9
:10152000860088D801E0B091BA00B35009F405E014
:10153000B0919600B01708F069CFF89491D890D880
:101540008FD8789479D820926A0020926B002092EC
:101550006C00B0916B00B395B0936B00BF3F71F519
:10156000B0916C00B395B0936C00B091CC0009E1E0
:10157000BA9559F002E3BA9541F00DE7BA9529F012
:101580000AEFBA9511F020926C00B0916C00B01780
:10159000A8F087DD47D8B0916C00BA95B0936C0085
:1015A00020926B00B091CB00B093AD00F89458D866
:1015B0007894B091CA00B093AD003CD837D8B091C0
:1015C0006800BB2319F485FF01C084CE01E085FDCE
:1015D00001C006E0B0919600B01708F4BACFB09100
:1015E000BA00B35009F026D8B0916800BB2309F4C3
:1015F00071CEF89456DD2092610020926200209214
:101600006300522C209264002092A1007894B09143
:10161000B700BB0FB0939F0020927E0020927F0006
:101620002092800020928100209282002092AA00C5
:1016300060E070E020927100B8E0B093AA007061A1
:10164000F1D7B2E074FDB1E0B7B9B6B1B068B0643B
:10165000B6B9B6B1B6FDFDCF04B115B1B6B1BF771D
:10166000B6B9112309F00FEF0093AB006CD9B8E0C5
:10167000B093AA00706165DDF894BFEFB0939B0052
:10168000ABD9B0916100B0939B00B0939C00B09334
:101690009D007894B1E0B0936100B09363005B2E3D
:1016A000B0936400B093A400B0919A00B093A300EB
:1016B000B091BA00B33019F49F7D87FD90627160DC
:1016C000726020926D0096DCACDC9FD9A4D99DD9C4
:1016D000A2D99BD910DB46D8B2DBE0DB9CD904DB76
:1016E00065FD41D877FFF9D877FD1BD9A8DBEDDB85
:1016F00092D901DB65FD59D8A2DB26DC8CD9F4DA5E
:1017000065FD8DD89CDB37DC86D9F5DA65FDB7D869
:1017100096DB70DC80D9E8DAB2E074FDB1E0B7B9ED
:10172000B6B1B068B064B6B98ADB7BDC74D90BD9CA
:1017300071FF21C0B0919E00B0939B00B0939C00BC
:10174000B0919A00B093A300B1E0B093A40018E167
:101750002CE0B0916D00B11740F07D7F7460209354
:101760006F00BFEFB0939B0006C0B0919600B13000
:1017700008F0B0CF64C072FF15C066FD13C0B09111
:101780006F00BA9519F47B7F7860A4CFB0936F0097
:10179000B0919600B13008F09DCFB091BA00B3304F
:1017A00009F04DC020927000B091990002E81091AC
:1017B000D600112309F003E0B01708F040C085FF00
:1017C00004C0B0916800BB23D1F1B091BA00B3302E
:1017D00081F495FD03C087FD04C00BC087FF01C0E5
:1017E00008C066FD06C06064B0919E00B0939B0087
:1017F00086CF00EF66FF05C0B0919E00B0939B00BE
:1018000000E2B0917B00B01708F464CF66FF17C008
:101810006F7B9F7D87FD90627460B2E1B0936F0033
:10182000B0919E00B0939B0055CFB0917000B395DE
:10183000B0937000B0919600BB2309F002C02092D3
:101840007000F8942EDC8090B900B2E0B093B9003B
:1018500078DC8092B9002092610020926200209290
:101860006300522C2092640020929F0060E070E0A0
:101870007894E0D616DC0091D600002319F0959AF2
:10188000AC9AC09AB6B1B460B6B985FF05C0B09144
:101890007000B43008F01ECD58CEEDE0F0E023D05B
:1018A0000A3509F01BC0EEE0F0E01DD0053A09F062
:1018B00015C03AE0A2EBB0E0E3E0F0E014D00D9305
:1018C00031963A95D9F739E1AEEBB0E0EFE0F0E0D0
:1018D0000AD00D9331963A95D9F702C0EFDB0AD0C2
:1018E000E8E2F0E00895E199FECFEEBBFFBBE09A9D
:1018F0000DB308951ED03AE0A2EBB0E0E3E0F0E0D3
:101900000D910FD031963A95D9F739E1AEEBB0E0B1
:10191000EFE0F0E00D9105D031963A95D9F712D06D
:101920000895E199FECF0DBBEEBBFFBBE29AE19AB1
:101930000895EDE0F0E00FEFF4DFEEE0F0E00FEF00
:10194000F0DF0895EDE0F0E00AE5EBDFEEE0F0E037
:1019500005EAE7DF08953091AE000091AF00313025
:1019600011F40093B600323011F40093B700333015
:1019700011F40093B800343011F40093C4003530F2
:1019800011F40093B900363011F40093D5003730CC
:1019900011F40093CE00383011F40093BA003930BE
:1019A00011F40093BB00089525E046D62A95E9F787
:1019B00008954DD64FD651D653D638D648D64AD6A6
:1019C0004CD64ED633D643D645D647D649D60895BB
:1019D00047D643D63FD63BD629D642D63ED63AD670
:1019E00036D624D63DD639D635D631D60895809010
:1019F000AE009090AF002BD62AD629D617D68A945F
:101A0000D1F72ED613D69A94E1F70895F894D1DF42
:101A10007894CADFC9DFB1E0B093AE00B1E0B09313
:101A2000AF002092B000F894E2DF7894B5E06B2E1E
:101A30007090960001D6B09196007B16C9F7B13030
:101A400018F0BF3F40F107C086DFF89453DFB1DFE5
:101A5000B8E0B1BDA9DF6A9459F7B091B000B39571
:101A6000B093B000B33008F4DECF9EDFB091AF008A
:101A7000B395B093AF00F894B091AE00BA95EEE391
:101A8000F0E0EB0FF21D049178940395B091AF0054
:101A9000B01708F4C6CF88DF87DFB091AE00B395EA
:101AA000B093AE00B091AE00BA3008F4B7CF06DB09
:0C1AB000F89420DFB8E0B1BD77DFC5CBB3
:00000001FF
